:020000040800F2
:100000009817002089010008910100089301000859
:100010009501000897010008990100080000000000
:100020000000000000000000000000009B0100082C
:100030009D010008000000009F010008A1010008C8
:10004000A3010008A3010008A3010008A301000800
:10005000A3010008A3010008A3010008A3010008F0
:10006000A3010008A3010008A3010008A3010008E0
:10007000A3010008A3010008A3010008A3010008D0
:10008000A3010008A3010008A3010008A3010008C0
:10009000A3010008A3010008A3010008A3010008B0
:1000A000A3010008A3010008A3010008A3010008A0
:1000B00081030008A3010008A3010008A3010008B0
:1000C000A3010008A3010008A3010008A301000880
:1000D000A3010008AF12000811140008A3010008D2
:1000E00041100008A3010008A301000800F002F875
:1000F00000F03AF80AA090E8000C82448344AAF188
:100100000107DA4501D100F02FF8AFF2090EBAE885
:100110000F0013F0010F18BFFB1A43F0010318473B
:100120001C3C00003C3C0000103A24BF78C878C159
:10013000FAD8520724BF30C830C144BF04680C60ED
:10014000704700000023002400250026103A28BF35
:1001500078C1FBD8520728BF30C148BF0B60704739
:100160001FB51FBD10B510BD03F05CFD1146FFF7B4
:10017000F7FF00F03EF903F08EFD03B4FFF7F2FF46
:1001800003BC00F093FF000009488047094800477E
:10019000FEE7FEE7FEE7FEE7FEE7FEE7FEE7FEE737
:1001A000FEE7FEE704480549054A064B7047000094
:1001B000FB380008ED000008981100209817002077
:1001C0009813002098130020F948006840F08070D0
:1001D000F74908600020F74948600846006840F089
:1001E000010008607047F3484068704710B500216F
:1001F0004FF0006001F069FA4FF4A06001F02EFAB0
:1002000010BD08B501211C2001F040FE0121084667
:1002100001F03CFE4FF40050ADF8000003208DF8D3
:10022000020010208DF803006946E34801F072FBDC
:100230004020ADF8000003208DF8020010208DF85A
:1002400003006946DD4801F065FB4021DB4801F011
:1002500010FC4FF48050ADF8000003208DF8020030
:1002600010208DF803006946D44801F053FB0121AA
:10027000082001F00BFE4FF46070ADF8000048203C
:100280008DF803006946CD4801F044FB08BD10B568
:100290000121084601F0FAFDC948406840F00070AD
:1002A000C749486010BD7FB505460C460121084688
:1002B00001F0F9FDADF80850ADF804400020ADF8AC
:1002C0000A00ADF8060001A94FF0804001F016FFCA
:1002D00001221146900702F088FA4FF4A06001F065
:1002E000BDF91C208DF8000000208DF801000320CE
:1002F0008DF8020001208DF80300684601F0B3F983
:100300000121880702F056FA7FBD10B5AD4800689C
:1003100040B1AC480838006820B1AA48001F006806
:10032000002829D1A8480078002828D10120A64912
:100330000870A448006830B90120A4490870A4A03E
:1003400003F05EFB1BE09F48001F006848B9A2A0B5
:1003500003F056FB02209D4908700020A049087058
:100360000DE098480838006848B99EA003F048FBA3
:1003700000209649087002E000209349087010BDE3
:1003800010B50121880702F0DEFCB8B1FFF7BDFF10
:100390008E480078002811DD94480088401C80B207
:1003A000924908800A2809DD9148006880F0010020
:1003B0009049C1F8B40100208C49088001218807C8
:1003C00002F0D2FC10BD70B58B4D6D6945F0010592
:1003D000894E7561642400BF251EA4F10104FBD180
:1003E0000C468460C2604360056845F09005056076
:1003F00070BD0024002081490870FFF7E5FE482009
:1004000000F076FDFFF7FDFEFFF7F0FE00F07CFE4A
:100410004FF4E13001F08DF84FF4E13000F079FF56
:100420004021774802F04EFE75481430008840F0B5
:1004300080007349143108800023724A7049091DF5
:100440007148FFF7C0FF642000F06EFD4FF47A7032
:1004500000F06AFD4FF47A7000F066FD4FF47A7098
:1004600000F062FD2221002000F0D6FAB0B967A0AA
:1004700003F0C6FA11E04FF400514F4801F0F7FACB
:100480004FF47A7000F050FD4FF400514A4801F0EB
:10049000F0FA4FF47A7000F047FDECE761A003F04A
:1004A000AFFA4FF40051444801F0E3FAC82000F0DD
:1004B0003BFD4FF40051404801F0D9FAC82000F04C
:1004C00033FD4FF400513C4801F0D1FA00F070F9CF
:1004D00041F61F416320FFF7E6FE40E03B4800780D
:1004E00001280CD10020564908704FF400513248C1
:1004F00001F0BFFA2221002000F05DFC2FE033481C
:100500000078022828D136480078C0B90A2000F0C7
:100510000BFDAA204B49087010204871AF2088714C
:10052000002048708870C87008710721454800F0A5
:1005300056FFC82000F0F8FC01202949087000206F
:1005400000F07CF9C0F30714204600F036FF4FF4AA
:10055000C87000F005FD02E0002025490860BDE7F5
:10056000F0B58BB006460C4615461F46224840693A
:1005700040F0010020494861234803F025F8009429
:100580000195102002900A20039000200490802002
:10059000059000200690079008904FF48050099035
:1005A00000200A906946304603F0B0F80BB0F0BD69
:1005B000FCED00E0001000E000100140000C0140E4
:1005C0000000014024812142040000200500002099
:1005D0006B6579310D0A00006B6579320D0A0000F8
:1005E0000E0000206B6579330D0A0000100000201A
:1005F000B4012242000022420010024030000020DC
:10060000004400407C040020440002400D0A436185
:100610006D65726120496E6974206661696C210D97
:100620000A0000000D0A43616D65726120496E6920
:10063000742053756363657373210D0A0000000015
:1006400003000020060000202DE9F04707468946F8
:100650001646B88900F4005010B90020BDE8F087B4
:100660005048384460B1B0F5806F05D0B0F5744F94
:100670000AD100254C4C07E002254B4C283C03E0F6
:100680000125494C3C3400BF00BFB6F5806F01D94D
:100690004FF480666068C8B905EBC510434941F85E
:1006A000306005EBC511414A02EBC10101F10800C0
:1006B0003246494603F0C2F9206820F0010020606C
:1006C0006660206840F00100206068E0C6F5806048
:1006D0006168A0EB010804E0C6F580606168A0EBEA
:1006E0000108B8F1000FF7DD206820F0010020605C
:1006F00005EBC5102D4951F830006168401A05EB33
:10070000C5112A4A02EBC1014860606805EBC511BA
:1007100042F8310005EBC51394460CEBC3030833D4
:1007200005EBC51C92460AEBCC0CDCF804C003EBCD
:100730000C0105EBC51394465CF8332005EBC5139B
:100740000CEBC30303F1080003F078F905EBC511C6
:10075000524602EBC101083105EBC512534653F86E
:10076000322088183246494603F068F905EBC51077
:10077000514651F83000304405EBC511524642F85D
:100780003100206820F00100206005EBC510114603
:1007900051F830006060206840F0010020600120C6
:1007A0005CE7000000BCFFBF44000240740400206E
:1007B00000B587B001214FF4017001F067FB4FF4E1
:1007C000004001F0C7FA0120ADF8180000208DF8B4
:1007D0001B0003208DF81A0006A9244801F09AF89E
:1007E000002001908DF808008DF809004FF460207A
:1007F00003900020049001208DF8140001A91C48EA
:1008000002F0E1FC01211A4802F009FD184802F04B
:1008100028FD00BF164802F029FD0028FAD114482F
:1008200002F02EFD00BF124802F02FFD0028FAD181
:1008300001210F4802F033FD07B000BD10B504469A
:100840000723012221460A4802F055FD01210848EC
:1008500002F025FD00BF0221054802F091FE0028AC
:10086000F9D0034802F0AEFD10BD000000080140C1
:10087000002401402DE9F04705460F4690461C46EE
:10088000DDE9089A0A9E1021F94803F01CF9F9489D
:10089000002101608180817142463946284603F07B
:1008A000CDF852464946204603F0C8F86E7066708F
:1008B000BDE8F08770B504460D462946204600F095
:1008C0006CFE70BD70B504460D460026EA4A294606
:1008D000204600F070FE0646304670BD2DE9FC4112
:1008E0000746884615461E46002000900190414666
:1008F0003846FFF7DFFF05216846FFF7E3FF10B931
:100900000020BDE8FC81002408E01DF80400295DFA
:10091000884201D00020F4E7601CC4B2B442F4DB8A
:100920000120EEE7FEB505460C460520D349D14B24
:100930000922CDE901050091D149CD48FFF79AFF81
:10094000362C01DDCA4804720523CA4A0921C84869
:10095000FFF7C4FF06463046FEBD3EB50446042000
:10096000C849C44B0246CDE901040091C649C048BC
:10097000FFF780FF0423BF4A1946BD48FFF7AEFFCB
:10098000054628463EBDFEB504460D460520BF4936
:10099000B84B0922CDE901040091BD49B448FFF7E5
:1009A00069FFB34805720523B24A0921FFF796FF94
:1009B00006463046FEBD70B586B005460E460020A0
:1009C000049005900620B349AA4B0822CDE9010501
:1009D0000091B149A648FFF74DFF0821A448FFF751
:1009E00069FF062104A8FFF76DFF10B9002006B0CB
:1009F00070BD002409E004A8005D9E49095D88429D
:100A000001D00020F3E7601CC4B2052CF3DB9DF895
:100A1000150030700120EAE7F8B505460C46FF20C6
:100A20000090362669462846FFF7C5FF28B9002101
:100A30009AA000F023FC0020F8BD9DF8000084423D
:100A400019D021462846FFF79EFF28B900219AA019
:100A500000F014FC0020EFE72846FFF77EFF28B9DE
:100A600000219CA000F00AFC0020E5E74FF47A701A
:100A700000F05AFA00949DF8000084420DD19DF8D0
:100A8000000030B1112802D0222804D100BF362640
:100A900002E0602600E000BF00BF31462846FFF7B5
:100AA00041FF28B900218FA000F0E8FB0020C3E738
:100AB000642000F039FA0120BEE73EB50446052067
:100AC00090496C4B0246CDE9010400918E4968487B
:100AD000FFF7D0FE0523674A19466548FFF7FEFE7B
:100AE000054628463EBD3EB5044605208749614B74
:100AF0000246CDE90104009185495D48FFF7BAFE41
:100B000005235C4A19465A48FFF7E8FE0546284681
:100B10003EBD70B586B0054607207E49554B05227F
:100B2000CDE9010500917C495148FFF7A3FE05215D
:100B30004F48FFF7BFFE092103A8FFF7C3FE10B916
:100B4000002006B070BD002409E003A8005D4949FB
:100B5000095D884201D00020F3E7601CC4B2072C75
:100B6000F3DB9DF8130006029DF81400064330469F
:100B7000E7E72DE9FE4307460D4616469946002451
:100B8000A046052065493B4B1022CDE901090091A3
:100B900063493748FFF76EFE380A354908724F72CD
:100BA000280A08734D7310213148FFF783FE05F1C1
:100BB0000A0081B23046FFF785FE10B90020BDE87B
:100BC000FE83002408E0305D2A49095D884201D097
:100BD0000020F4E7601CC4B2052CF4DB00240AE01A
:100BE000601D2844305C2349095D884201D0002003
:100BF000E5E7601CC4B2052CF2DBB04607E098F8CC
:100C0000050088F80000681E85B208F10108002D73
:100C1000F5DC0120D3E73EB5044605204149154BDC
:100C20000922CDE9010400913F491148FFF722FE56
:100C30000523104A09210E48FFF750FE05462846B5
:100C40003EBD3EB50446052038490A4B0246CDE973
:100C50000104009136490648FFF70CFE0523054ABA
:100C600019460348FFF73AFE054628463EBD0000F8
:100C70007C0800201C00002040420F00F63C0008C9
:100C8000ED3C0008B03C0008B43C0008043D0008FE
:100C9000FB3C0008113D0008093D00080D0A726583
:100CA00061645F70686F746F5F73697A65206572E5
:100CB000726F720D0A0000000D0A7365745F706830
:100CC0006F746F5F73697A65206572726F720D0A57
:100CD000000000000D0D65736574206572726F72FF
:100CE0000D0A00000D0A73656E645F636F6D7072AC
:100CF0006573735F72617465206572726F720D0A3D
:100D000000000000BD3C0008B83C0008C73C0008DB
:100D1000C23C0008D13C0008CC3C0008E83C00087C
:100D2000D83C0008343D00082B3D0008213D000858
:100D3000173D00083EB5044605206449644B024651
:100D4000CDE90104009163496348FFF793FD052352
:100D50005F4A19466048FFF7C1FD054628463EBD7B
:100D60001CB5044600200090019005216846FFF75D
:100D7000A9FD08B900201CBD9DF80000574909785D
:100D8000884211D19DF802005449897888420BD1DC
:100D90009DF803005149C978884205D19DF80400A7
:100DA0004E490979884201D00020E4E79DF801000E
:100DB00020700120DFE72DE9F04105468846002636
:100DC0000027002441462846FFF726FE44490870C4
:100DD0000846007810B90020BDE8F0812846FFF7EA
:100DE0006CFE08B90020F7E72846FFF77CFE08B93B
:100DF0000020F1E72846FFF78CFE3A4908600846D4
:100E0000006808B90020E7E736480068C0F38F267D
:100E100034480088C0F30907AA2033490870052028
:100E20004871AF2088712F480068000E48702D4827
:100E30000068000C88702B480088000AC870294898
:100E4000007808710721284800F0C9FA642000F0F2
:100E50006BF8FEB100241BE04FF40061234802F060
:100E600032FE4FF6FF7101EA84202B461F4A4FF4F1
:100E70008061FFF77EFE08B90020ADE74FF4806186
:100E80001A4800F0ACFA322000F04EF8601C84B230
:100E9000B442E1DBBFB14FF40061144802F013FE2D
:100EA0004FF6FF7101EA84202B46104A3946FFF7BE
:100EB00060FE08B900208FE739460C4800F08FFA31
:100EC000322000F031F8012086E70000213D0008C3
:100ED0001C0000201C3D00087C080020263D000866
:100EE000140000201800002024000020F00800203A
:100EF0004FF0E021096921F004014FF0E022116177
:100F0000C21700EB5272C2F3C702294B1A7019467E
:100F1000097801EB4102C2EBC1114FF6FF7202EA00
:100F2000C101244A118070470146224A12884A436F
:100F30004FF0E0235A6100229A6101221A6100BF3A
:100F40004FF0E022106900F001021AB100F4803283
:100F5000002AF5D000224FF0E0231A619A61704711
:100F60000146134A12784A434FF0E0235A610022A7
:100F70009A6101221A6100BF4FF0E022106900F06F
:100F800001021AB100F48032002AF5D000224FF09D
:100F9000E0231A619A61704710B5044603E04FF4EC
:100FA0007A70FFF7C1FF201EA4F10104F7D110BD34
:100FB0002C0000202E0000201FB50121112000F080
:100FC00065FF4FF40040ADF80C0048208DF80F008D
:100FD00003A9324800F09EFC0F21022000F0B0FD72
:100FE0004FF40040019000208DF808000C208DF88F
:100FF000090001208DF80A0001A800F0ABFB2820B1
:101000008DF8000001208DF801008DF802008DF8A8
:101010000300684600F027FB1FBD10B54FF40040E9
:1010200000F00FFC1E48006840F400401C490860B6
:1010300010BD1B48006820F4004019490860704743
:1010400010B54FF4004000F0EBFB40B16420FFF717
:101050006BFF012013490870C00300F0F2FB10BDC4
:1010600010B50F48006820F400400D4908600022C8
:1010700040F225510C4801F056FF10BD10B540F26A
:101080002551094802F05EF8012240F22551064838
:1010900001F049FFFFF7C1FF10BD00000010014043
:1010A000000401403000002000440040014600BF21
:1010B000704770B5044600250020F8490860682094
:1010C000FFF74EFF00BF0EE004F0010018B1012051
:1010D000F249086002E00020F04908606820FFF74C
:1010E0003FFF64106D1C082DEEDB0120EB4908600A
:1010F0006820FFF735FF70BD70B504460D46E0B2BD
:10110000FFF7D7FF204670BD1CB5012144F2050052
:1011100000F0BCFE4FF40070ADF8040018208DF80C
:10112000070003208DF8060001A9DD4800F0F2FB5E
:101130004FF48060ADF8040004208DF8070001A989
:10114000D74800F0E7FB25208DF8000001208DF83E
:1011500001008DF802008DF80300684600F083FA64
:101160000121480400F09FFE0420ADF8040018207F
:101170008DF8070003208DF8060001A9C84800F08B
:10118000C9FB0820ADF8040004208DF8070001A970
:10119000C34800F0BFFB26208DF8000001208DF829
:1011A00001008DF802008DF80300684600F05BFA3C
:1011B0001CBD10B586B00446012144F2040000F0C5
:1011C00065FE4FF40070ADF8140003208DF8160092
:1011D00018208DF8170005A9B14800F09BFB4FF4CB
:1011E0008060ADF8140004208DF8170005A9AC4804
:1011F00000F090FB25208DF8000001208DF8010003
:1012000003208DF8020001208DF80300684600F0ED
:101210002AFA01940020ADF80800ADF80A00ADF8F4
:101220000C00ADF810000C20ADF80E0001A99D488F
:1012300001F0E1FD012240F225519A4801F073FED0
:10124000012240F22441974801F06DFE01219548AA
:1012500001F05DFE06B010BD10B504464021914876
:1012600001F03DFF21468F4801F0BEFE00BF402146
:101270008C4801F027FF0028F9D010BD70B5054655
:101280000E4656B9002404E0285DFFF712FF601CEB
:1012900084B2285D0028F7D108E0002404E0285D2E
:1012A000FFF707FF601C84B2B442F8D370BD70B57D
:1012B000002540F225517B4801F01AFFC0B1794862
:1012C00001F096FEC4B278480068132808D2764828
:1012D00001680068401C744A10607448445402E07D
:1012E00000207149086040F225516E4801F02AFF44
:1012F00040F224416B4801F0FBFE48B16948008888
:10130000C5B26848001D0088C5B200206649086063
:1013100070BD10B586B004460121480400F0C3FD3D
:101320000121042000F0B2FD0420ADF814000320D8
:101330008DF8160018208DF8170005A9584800F000
:10134000E9FA0820ADF8140004208DF8170005A96B
:10135000534800F0DFFA01940020ADF80800ADF822
:101360000A00ADF80C00ADF810000C20ADF80E002E
:1013700001A94F4801F03FFD26208DF80000022012
:101380008DF8010003208DF8020001208DF8030084
:10139000684600F068F9012240F22551444801F006
:1013A000C2FD012240F22441414801F0BCFD01216F
:1013B0003F4801F0ACFD06B010BD10B50446402119
:1013C0003B4801F08CFE2146394801F00DFE00BF7C
:1013D0004021374801F076FE0028F9D010BD70B5E5
:1013E00005460E464EB1002404E0285DFFF7E5FFF8
:1013F000601C84B2B442F8D309E0002404E0285D04
:10140000FFF7DBFF601C84B2285D0028F7D170BDB8
:1014100010B5002440F22551254801F069FEA0B125
:10142000234801F0E5FDC4B222480068312808D203
:10143000204801680068401C1E4A10601E48445441
:1014400076E000201B49086072E040F22441184811
:1014500001F04EFE00286BD015480088C4B2144835
:10146000001D0088C4B21348006800285CD000202A
:10147000104908601148007838B911A10E4802F0EF
:10148000CBFA10B101200D49087010A10A4802F0F2
:10149000C3FA08B301200F49087038E0B081214237
:1014A000000801400038014038000020F010002002
:1014B00000440040400000200411002049000020AA
:1014C000534D53205245414459000000434F4E4E66
:1014D000454354004800002055A1574802F09CFAAB
:1014E000A8B1002055490870012080F3138800BF7F
:1014F00000BF5348006800F4E06052490843001DF3
:101500004F490860BFF34F8F00BF00BFFEE74EA1F9
:10151000494802F081FA10B101204E490870322189
:10152000454802F0D0FA03E03221434802F0CBFAFA
:1015300010BD1FB5044600940020ADF80400ADF8BE
:101540000600ADF80800ADF80C000C20ADF80A005C
:101550006946414801F04FFC01213F4801F0D7FCAA
:10156000002240F225513C4801F0DDFC40213A4880
:1015700001F0B5FD1FBD10B504464021364801F00D
:10158000AEFD2146344801F02FFD00BF4021324816
:1015900001F098FD0028F9D010BD70B506460D4643
:1015A00045B1002404E0305DFFF7E5FF601C84B224
:1015B000AC42F8D370BD2DE9F04106460F46904687
:1015C00000240025244801F013FD044608E0012012
:1015D000FFF7C6FC6D1C454502D90020BDE8F0812F
:1015E00020211D4801F06EFD0028F0D01A4801F0BE
:1015F000FFFC30700124002515E02021164801F081
:1016000061FD50B10025144801F0F2FC3055601C1A
:1016100084B2BC4207D137B106E042F21070854275
:1016200000D901E06D1CE8E700BF2046D6E70000C6
:10163000434C4F5345000000041100204800002097
:101640000CED00E00000FA0543616D5F53746172B8
:1016500074000000030000200038014031490143BC
:10166000314A1160704770B5002100230F22C47801
:1016700004B32D4C246804F4E064C4F5E064210A4A
:10168000C1F10403CA40447804FA03F18478144099
:1016900021430901254C0678A155047804F01F0563
:1016A0000124AC4005786D11AD0005F1E025C5F8C9
:1016B000004109E0047804F01F050124AC401C4DF2
:1016C0000678761145F8264070BD1A4A0A40024352
:1016D000154B1B1F1A60704739B1134A121D12684F
:1016E0000243114B1B1D1A6006E00F4A121D1268BF
:1016F00082430D4B1B1D1A607047042808D14FF020
:10170000E021096941F004014FF0E022116107E096
:101710004FF0E021096921F004014FF0E02211614E
:10172000704700000000FA050CED00E000E400E066
:1017300080E100E080FFFF1F002044490860091D90
:101740000860091D0860091D086041483F491431BF
:101750000860704700213D498279002A3AD00A4644
:10176000126803689A430B461A600A1D12680368E0
:101770009A430B1D1A60027911440A6803681A43E0
:101780000A60324A0832126803689A432F4B0833C2
:101790001A601A1D126803689A432C4B0C331A60A6
:1017A0004279102A0ED11A1F126803681A43274B78
:1017B00008331A601A1D126803681A43234B0C334E
:1017C0001A600DE02149427911440A6803681A43FE
:1017D0000A6005E0027911440A6803689A430A60C6
:1017E00070470021016001710C214171002181715C
:1017F00070471649103109680143144A10321160CC
:10180000704701460020114A143212680A400AB19A
:10181000012000E0002070470C4914310860704737
:10182000014600200022094B1B6803EA0102074B16
:1018300014331B680B4013B10AB1012000E00020F3
:1018400070470249143108607047000000040140ED
:10185000FFFF0F0010B50446CC48844208D1012197
:10186000042000F02DFB0021042000F029FB46E0BD
:10187000C748844208D10121082000F021FB002143
:10188000082000F01DFB3AE0C248844208D1012143
:10189000102000F015FB0021102000F011FB2EE0BD
:1018A000BD48844208D10121202000F009FB00211D
:1018B000202000F005FB22E0B848844208D1012135
:1018C000402000F0FDFA0021402000F0F9FA16E077
:1018D000B348844208D10121802000F0F1FA0021B0
:1018E000802000F0EDFA0AE0AE48844207D10121E1
:1018F000801500F0E5FA0021A01500F0E1FA10BD16
:1019000010B50121084600F0DBFA0021012000F0AB
:10191000D7FA10BD2DE9F04102460025002600202F
:1019200000230024002791F803C00CF00F0591F864
:1019300003C00CF0100CBCF1000F03D091F802C0F2
:101940004CEA050591F800C0BCF1000F31D01468D5
:1019500000202BE04FF0010C0CFA00F3B1F800C0AE
:101960000CEA03069E4220D183004FF00F0C0CFAC4
:1019700003F7BC4305FA03FC4CEA040491F803C0E6
:10198000BCF1280F06D14FF0010C0CFA00FCC2F894
:1019900014C00AE091F803C0BCF1480F05D14FF024
:1019A000010C0CFA00FCC2F810C0401C0828D1D36E
:1019B0001460B1F800C0BCF1FF0F34DD54680020A2
:1019C0002EE000F1080C4FF0010808FA0CF3B1F812
:1019D00000C00CEA03069E4221D183004FF00F0C99
:1019E0000CFA03F7BC4305FA03FC4CEA040491F833
:1019F00003C0BCF1280F05D100F1080C08FA0CF85F
:101A0000C2F8148091F803C0BCF1480F07D100F16F
:101A1000080C4FF0010808FA0CF8C2F81080401CBE
:101A20000828CED35460BDE8F0814FF6FF710180E5
:101A3000022181700421C170704702460020936822
:101A40000B400BB1012000E0002070470146886880
:101A500080B2704702460020D3680B400BB10120D2
:101A600000E0002070470146C86880B270470161FD
:101A70007047416170470AB1016100E04161704700
:101A8000C16070474FF480320A4382618161826194
:101A900082698269704702460020434B18684FF6FE
:101AA0008073184040EA021008433F4B18607047AB
:101AB0003E49C8617047F0B50A4600230024002162
:101AC000002500F00046B6F1004F02D1364EF16914
:101AD00001E0354E7168C0F3034583B200F440164F
:101AE000B6F5401F08D121F070612F4E766826F0C0
:101AF00070662D4F7E6012E000F48016B6F5801FF0
:101B000006D1032606FA05F4A14341F0706106E010
:101B1000460D360103FA06F6B14341F0706122B179
:101B2000460D360103FA06F6314300F00046B6F1E1
:101B3000004F02D11C4EF16101E01B4E7160F0BDFF
:101B400030B500228B071C0F0F2303FA04F2164B4B
:101B500008338C1053F824309343134C08348D1001
:101B600044F8253023468C1053F824308C07240F7A
:101B700000FA04F423430C4C08348D1044F825304B
:101B800030BD0A49DC3108607047000000080140A0
:101B9000000C0140001001400014014000180140F9
:101BA000001C0140002001400000014000002042D4
:101BB000DF48006840F00100DD49086008464068E1
:101BC000DC490840DA49486008460068DA490840BC
:101BD000D74908600846006820F48020086008465D
:101BE000406820F4FE0048604FF41F008860704792
:101BF000CF49096821F48031CD4A11601146096846
:101C000021F480211160B0F5803F03D0B0F5802F22
:101C10000ED106E0C649096841F48031C44A11601A
:101C200007E0C349096841F4A021C14A116000E0FE
:101C300000BF00BF704710B50146002200230020FE
:101C40004A11012A02D1BA4C236806E0022A02D1C5
:101C5000B74C236A01E0B64C636A01F01F0201240D
:101C600094401C400CB1012000E0002010BD38B5AC
:101C7000002000900024002500BF3120FFF7DBFF8B
:101C800005460098401C00900098B0F5A06F01D068
:101C9000002DF2D03120FFF7CEFF08B1012400E083
:101CA0000024204638BD01460020A14A106820F0DB
:101CB000F80040EAC10010607047A0490860704712
:101CC000024600209A4B586820F47C1042EA010337
:101CD0001843974B5860704798490866704701460B
:101CE0000020934A506820F003000843506070477A
:101CF0008F48406800F00C007047014600208C4A75
:101D0000506820F0F0000843506070470146002002
:101D1000874A506820F4E0600843506070470146ED
:101D20000020834A506820F4605040EAC1005060AF
:101D3000704729B17E4A527A02437D4B5A7204E0C1
:101D40007B4A527A82437A4B5A7270477B49D83128
:101D50000860704701460020754A506820F44040F2
:101D60000843506070470021714A20321170704A58
:101D700082F82010012802D004280AD104E00121B1
:101D80006B4A2032117005E00521694A203211703A
:101D900000E000BF00BF70476949086070476449B0
:101DA000096A0143624A1162704765494439086013
:101DB000704730B500210022002400235C4D6D687F
:101DC00005F00C0121B1042905D0082923D105E033
:101DD0005C4D056022E05B4D05601FE0544D6D6871
:101DE00005F47012524D6D6805F48034022505EB40
:101DF00092421CB9544D554305600BE04C4D6D6843
:101E000005F400351DB1504D5543056002E04D4DC0
:101E10005543056002E04B4D056000BF00BF444DD7
:101E20006D6805F0F0010909484D6B5C0568DD40FF
:101E300045603F4D6D6805F4E061090A434D6B5CF8
:101E40004568DD4085603A4D6D6805F46051C90A0A
:101E50003E4D6B5C4568DD40C560354D6D6805F4F1
:101E60004041890B3A4D6B5CC568B5FBF3F50561E4
:101E700030BD29B12E4A526902432D4B5A6104E00C
:101E80002B4A526982432A4B5A61704729B1284A2A
:101E900092690243264B9A6104E0254A9269824383
:101EA000234B9A61704729B1214AD2690243204BE2
:101EB000DA6104E01E4AD26982431D4BDA61704741
:101EC00029B11B4AD2680243194BDA6004E0184A70
:101ED000D2688243164BDA60704729B1144A1269FE
:101EE0000243134B1A6104E0114A12698243104BFA
:101EF0001A61704712494039086070470F49C86439
:101F000070470B49C87170470948406A40F08070BB
:101F100007494862704701460020054A92680A4016
:101F20000AB1012000E00020704701498872704723
:101F3000001002400000FFF8FFFFF6FE00004242E2
:101F40008004424200127A0000093D004A0000204D
:101F50005A00002010B50446FE48844208D10121F1
:101F6000C014FFF7ADFF0021E014FFF7A9FFC4E0A4
:101F7000B4F1804F08D101210846FFF7AEFF0021E0
:101F80000120FFF7AAFFB8E0F348844208D10121FD
:101F90000220FFF7A2FF00210220FFF79EFFACE026
:101FA000EE48844208D101210420FFF796FF00216A
:101FB0000420FFF792FFA0E0E948844208D1012104
:101FC0000820FFF78AFF00210820FFF786FF94E032
:101FD000E448844208D101211020FFF77EFF002150
:101FE0001020FFF77AFF88E0DF48844208D1012102
:101FF0002020FFF772FF00212020FFF76EFF7CE01A
:10200000DA48844208D101214014FFF759FF00212A
:102010006014FFF755FF70E0D548844209D10121D3
:10202000C804FFF74DFF00214FF40020FFF748FFE1
:1020300063E0D048844209D101210805FFF740FF41
:1020400000214FF48010FFF73BFF56E0CA4884425E
:1020500009D101214805FFF733FF00214FF400109B
:10206000FFF72EFF49E0C548844208D101214020F6
:10207000FFF733FF00214020FFF72FFF3DE0C0486E
:10208000844208D101218020FFF727FF0021802012
:10209000FFF723FF31E0BB48844208D101218015BE
:1020A000FFF71BFF0021A015FFF717FF25E0B6483B
:1020B000844209D101210804FFF702FF00214FF4F7
:1020C0008030FFF7FDFE18E0B048844209D10121BD
:1020D0004804FFF7F5FE00214FF40030FFF7F0FE53
:1020E0000BE0AB48844208D101218804FFF7E8FEE9
:1020F00000214FF48020FFF7E3FE10BD002202888C
:10210000944B98420ED0994B98420BD0B0F1804F2F
:1021100008D0914B984205D0904B984202D0904BFA
:10212000984204D14FF68F731A404B881A438D4B57
:10213000984207D08C4B984204D04FF6FF431A4088
:10214000CB881A4302808B8883850B880385814B5B
:1021500098420BD0854B984208D08B4B984205D0C3
:102160008A4B984202D08A4B984201D10B7A03865F
:1021700001238382704770B5002400220023058C60
:102180004FF6FE7635400584028C8388048B4FF62B
:102190008F752C40B51E2C400D882C43751E2A408F
:1021A0000D892A434D882A436A4DA8420BD06F4DB2
:1021B000A84208D0744DA84205D0744DA84202D060
:1021C000734DA84213D14FF6F7752A404D892A4323
:1021D0004FF6FB752A408D882A434FF6FF652B404A
:1021E0004FF6FF552B408D892B43CD892B438380A0
:1021F0000483CD888586028470BD70B500240022DA
:102200000023058C4FF6EF7635400584028C8388D9
:10221000048B48F6FF752C404FF6FF452C400D8887
:102220004FF6FF7606EA05252C434FF6DF752A4068
:102230000D8906EA05152A434D8806EA05152A4345
:10224000444DA84202D0494DA8421DD14FF67F759A
:102250002A404D894FF6FF7606EA05152A434FF6C8
:10226000BF752A408D8806EA05152A434FF6FF35CB
:102270002B404FF2FF752B408D8906EA85052B43D5
:10228000CD8906EA85052B4383800483CD880587A5
:10229000028470BD70B5002400220023058C4FF627
:1022A000FF6635400584028C8388848B4FF68F75DA
:1022B0002C404FF6FC752C400D882C434FF6FF55F3
:1022C0002A400D894FF6FF7606EA05252A434D88F8
:1022D00006EA05252A431F4DA84202D0234DA842F5
:1022E0001DD14FF2FF752A404D894FF6FF7606EA61
:1022F00005252A434FF6FF352A408D8806EA052535
:102300002A434EF6FF752B404DF6FF752B408D8905
:1023100006EA05152B43CD8906EA05152B43838074
:102320008483CD888587028470BD70B50022002328
:102330000024058C4EF6FF7635400584038C848896
:10234000828B48F6FF752A404FF6FF452A400D88DC
:1023500020E00000002C0140000400400008004084
:10236000000C004000100040001400400034014008
:10237000004C014000500140005401400018004052
:10238000001C00400020004000400140004401408B
:10239000004801404FF6FF7606EA05252A434DF630
:1023A000FF752B400D8906EA05352B434D8806EA5B
:1023B00005352B43FA4DA84202D0FA4DA84208D168
:1023C0004BF6FF752C408D894FF6FF7606EA851592
:1023D0002C4384808283CD88A0F84050038470BD54
:1023E000828B4FF2FF331A408283828B4FF6FF734A
:1023F00003EA01231A4382837047F0B50C46154661
:10240000002200210026078C4EF6FF7C07EA0C070D
:102410000784828B018C4FF6FF7707EA043640F67B
:10242000FF473A404FF6FF7707EA05273A434FF652
:10243000FF7707EA03373A43D94FB8420ED0D94F56
:10244000B8420BD0B0F1804F08D0D74FB84205D07A
:10245000D64FB84202D0D64FB84206D14DF6FF77DC
:10246000394046F48057394305E047F6FF57394075
:1024700044F48057394382830184F0BD828B4FF648
:10248000F3731A408283828B0A4382837047F0B5CC
:102490000C461546002200210026078C4FF6FF6CE3
:1024A00007EA0C070784828B018C4FF6FF7707EA57
:1024B00004264FF60C773A404FF6FF7707EA0317EA
:1024C0002F433A43B64FB8420ED0B64FB8420BD066
:1024D000B0F1804F08D0B44FB84205D0B34FB842E6
:1024E00002D0B34FB84206D14FF6FF57394046F4F9
:1024F0008077394305E04FF2FF57394044F4807745
:10250000394382830184F0BD028B4FF2FF331A40BE
:102510000283028B4FF6FF7303EA01231A430283FF
:102520007047F0B50C461546002200210026078CA6
:102530004FF6EF7C07EA0C070784028B018C4FF6FD
:10254000FF7707EA041640F6FF473A404FF6FF7759
:1025500007EA03373A434FF6FF7707EA05273A437E
:102560008F4FB8420ED08F4FB8420BD0B0F1804F92
:1025700008D08D4FB84205D08C4FB84202D08C4F56
:10258000B84206D14FF6DF77394046F0100739439D
:1025900005E04FF65F77394044F010073943028376
:1025A0000184F0BD028B4FF6F3731A400283028B55
:1025B0000A4302837047F0B50C46154600220021FD
:1025C000068C4FF6FE773E400684028B018C4FF658
:1025D0000C7632407E1C06EA03162E433243704EC0
:1025E000B0420ED06F4EB0420BD0B0F1804F08D049
:1025F0006D4EB04205D06D4EB04202D06C4EB0422E
:1026000006D14FF6FD76314044F00106314305E036
:102610004FF6F576314044F00106314302830184E0
:10262000F0BD70B505460C465D4885420ED05D484C
:1026300085420BD0B5F1804F08D05B48854205D06C
:102640005A48854202D05A48854200D100E000BF76
:10265000208850B92389A28861882846FFF7ABFFFC
:10266000E1882846FFF79EFF25E0208804280AD14C
:102670002389A28861882846FFF753FFE18828460E
:10268000FFF742FF17E0208808280AD12389A28893
:1026900061882846FFF7FBFEE1882846FFF7EEFE3B
:1026A00009E02389A28861882846FFF7A6FEE18811
:1026B0002846FFF795FE70BD2DE9F04105460C4612
:1026C00000260127608808B9022600E00026A088BD
:1026D000012801D1022700E001272088A0B9238921
:1026E000A28861882846FFF766FFE1882846FFF741
:1026F00059FF23893A4631462846FFF712FFE18801
:102700002846FFF701FF13E02389A2886188284645
:10271000FFF707FFE1882846FFF7F6FE23893A46D0
:1027200031462846FFF747FFE1882846FFF73AFF82
:10273000BDE8F0810A884B881A438B881A43CB88FE
:102740001A430B891A434B891A438B891A43A0F801
:10275000442070474FF6FF71818000210180C180C5
:102760004180017270470021018041808180C180D9
:10277000018141818181C1817047002101804180B7
:10278000012181800021C1800181704700210180E9
:1027900041808180C1800181418181817047000039
:1027A000002C0140003401400004004000080040BB
:1027B000000C004021B1028842F00102028004E0D6
:1027C00002884FF6FE731A400280704731B1B0F8AC
:1027D000442042F40042A0F8442005E0B0F8442030
:1027E000C2F30E02A0F8442070471AB183890B434C
:1027F000838102E083898B438381704781827047A4
:1028000041EA0203A0F8483070471AB183890B43AC
:10281000838102E083898B438381704701894FF66E
:10282000F8721140018170470A46002101894FF674
:102830008F73194011430181704730B504460D462E
:1028400029462046FFF7F0FF208940F0070020814D
:1028500030BD2DE9F04104460D4616461F46602D59
:1028600006D13B46012231462046FFF75AFE05E0DD
:102870003B46012231462046FFF79DFE2946204671
:10288000FFF7D2FF208940F007002081BDE8F081EA
:1028900030B50C4600210189C9B24FF6FF7505EA33
:1028A0000325154325432943018130BD2DE9F0411E
:1028B00005460E4617469846002443463A4631469A
:1028C0002846FFF7E5FF2C894FF6F870044044F0E6
:1028D00007044FF68F70044044F070042C81BDE86B
:1028E000F081F0B504460D4616461F463B4632467B
:1028F00029462046FFF7CCFF208940F48040208104
:10290000F0BD0185828270470A46002101884FF69A
:102910008F731940114301807047F0B50C4615467E
:102920001E460021002200230189028B038C4FF6F2
:10293000F877394021434FF6FC473A4040F20117FF
:102940003A434FF6DD773B404FF6FF7707EA06172D
:102950002F433B43018102830384F0BD0A460021DB
:10296000018B4FF68F7319401143018370470A465C
:102970000021018B48F6FF7319404FF6FF7303EAFD
:1029800002231943018370470A460021818B4FF6C9
:102990008F7319401143818370470A460021818B50
:1029A00048F6FF7319404FF6FF7303EA02231943F9
:1029B0008183704721B1028842F08002028004E0E6
:1029C00002884FF67F731A400280704721B18288D7
:1029D00042F00402828004E082884FF6FB731A40C2
:1029E0008280704721B1828842F00802828004E030
:1029F00082884FF6F7731A408280704721B182882F
:102A000042F00102828004E082884FF6FE731A4091
:102A1000828070470A460021018B4FF6F7731940F8
:102A20001143018370470A460021018B4FF2FF7367
:102A300019404FF6FF7303EA0223194301837047DD
:102A40000A460021818B4FF6F773194011438183A9
:102A500070470A460021818B4FF2FF7319404FF6F1
:102A6000FF7303EA02231943818370470A4600215A
:102A7000018B4FF6FB7319401143018370470A46DF
:102A80000021018B4FF6FF3319404FF6FF7303EA25
:102A900002231943018370470A460021818B4FF6B8
:102AA000FB7319401143818370470A460021818BD3
:102AB0004FF6FF3319404FF6FF7303EA0223194321
:102AC000818370470A460021018B4FF67F731940BE
:102AD0001143018370470A460021018BC1F30E01A7
:102AE0004FF6FF7303EA02231943018370470A4636
:102AF0000021818B4FF67F7319401143818370470A
:102B00000A460021818BC1F30E014FF6FF7303EAE1
:102B100002231943818370470A460021018C4FF636
:102B2000FD7319401143018470470A460021018C4E
:102B30004FF6F77319401143018470470A4600218C
:102B4000018C4FF6DF7319404FF6FF7303EA02134F
:102B50001943018470470A460021018C4FF67F73A8
:102B600019404FF6FF7303EA0213194301847047BB
:102B70000A460021018C4FF6FF5319404FF6FF73B0
:102B800003EA02231943018470470A460021018C9D
:102B90004FF2FF7319404FF6FF7303EA0223194304
:102BA000018470470A460021018C4DF6FF731940DD
:102BB0004FF6FF7303EA023319430184704730B5BF
:102BC000002301248C40A3B2048C9C430484048C15
:102BD00002FA01F5ADB22C43048430BD30B50023B8
:102BE00004248C40A3B2048C9C430484048C02FA19
:102BF00001F5ADB22C43048430BD70B5034600200E
:102C000000241846183001258D40ACB21D8CA54318
:102C10001D8409B1082909D100EB6100056825F080
:102C2000700505600568154305600EE00D1FC5F3CE
:102C30004E052844056825F4E045056005684FF613
:102C4000FF7606EA02263543056070BD21B1028891
:102C500042F00202028004E002884FF6FD731A403F
:102C60000280704721B1028842F00402028004E031
:102C700002884FF6FB731A400280704721B18288A8
:102C800042F08002828004E082884FF67F731A400F
:102C90008280704702884FF6F7731A4002800288DC
:102CA0000A430280704782884FF68F731A408280F1
:102CB00082880A438280704702894FF6F8731A406F
:102CC000028102890A430281704702894FF67F73AD
:102CD0001A40028102890A43028170478184704749
:102CE000818570478186704701877047818770476B
:102CF000A0F84010704702884FF6FF431A40028048
:102D000002880A43028070470146888E7047014658
:102D1000088F70470146888F70470146B1F8400020
:102D200070470146888C70470146088D70470246FF
:102D30000020138A0B400BB1012000E000207047F7
:102D4000CA430282704730B50246002000230024A7
:102D5000158A05EA0103958905EA010413B10CB14E
:102D6000012000E0002030BDCA430282704700000D
:102D700010B50446FB48844209D101218803FFF7BE
:102D80009FF800214FF48040FFF79AF832E0F648B0
:102D9000844209D101214804FFF79FF800214FF434
:102DA0000030FFF79AF825E0F048844209D101216C
:102DB0008804FFF792F800214FF48020FFF78DF888
:102DC00018E0EB48844209D10121C804FFF785F8D7
:102DD00000214FF40020FFF780F80BE0E548844223
:102DE00008D101210805FFF778F800214FF4801081
:102DF000FFF773F810BD2DE9F04786B005460E4683
:102E00000024A24600BFA1460027B08900B100BF40
:102E10002F462C8A4CF6FF700440F08804432C8225
:102E2000AC894EF6F3100440B088318908437189AB
:102E300008430443AC81AC8A4FF6FF400440B0899C
:102E40000443AC8201A8FEF7B4FFC648874202D112
:102E5000DDF810A001E0DDF80CA0A88900F4004026
:102E600040B10AEBCA0000EB0A1031684900B0FB20
:102E7000F1F807E00AEBCA0000EB0A10316889009C
:102E8000B0FBF1F86420B8FBF0F0040120096421E4
:102E900001FB1089A88900F4004040B1322000EB0A
:102EA000C900B0FBF1F000F00700044308E0322055
:102EB00000EB09106421B0FBF1F000F00F000443B7
:102EC0002C8106B0BDE8F0874FF416510160002157
:102ED0008180C18001810C21418100218181704765
:102EE00010B502460020108A4FF2FF0318400B88ED
:102EF0004C8823438C882343CC8823431843108277
:102F000010BD0021018041808180C180704721B1C6
:102F1000828942F40052828104E082894DF6FF7377
:102F20001A4082817047F0B5034600240026002530
:102F3000002040F66A17B94200D100BF1846C1F31D
:102F4000421401F01F06012707FA06F5012C01D1F2
:102F50000C3004E0022C01D1103000E014301AB122
:102F600007682F43076002E00768AF430760F0BDC2
:102F70001AB1838A0B43838202E0838A8B43838264
:102F80007047028A4FF6F0731A400282028A0A439F
:102F90000282704782894FF2FF731A4082818289D0
:102FA0000A438281704721B1828942F00202828104
:102FB00004E082894FF6FD731A4082817047028ACD
:102FC0004FF6DF731A400282028A0A430282704778
:102FD00021B1028A42F48042028204E0028A4BF666
:102FE000FF731A4002827047C1F308028280704763
:102FF00001468888C0F308007047818941F00101CB
:1030000081817047028BD2B20283028B42EA012295
:1030100002837047028B02F47F420283028B0A43D1
:103020000283704721B1828A42F02002828204E04A
:10303000828A4FF6DF731A408282704721B1828AFA
:1030400042F01002828204E0828A4FF6EF731A4047
:103050008282704721B1828A42F00802828204E0B3
:10306000828A4FF6F7731A408282704721B18289B3
:1030700042F40042828103E08289C2F30E0282811F
:10308000704721B1828A42F40062828204E0828A1F
:103090004FF2FF731A4082827047828A4FF6FB73A9
:1030A0001A408282828A0A438282704721B1828AD0
:1030B00042F00202828204E0828A4FF6FD731A40D7
:1030C0008282704702460020B1F5007F00D100BF28
:1030D00013880B400BB1012000E00020704701F481
:1030E0000072B2F5007F00D100BFCA430280704772
:1030F00070B50246002400230025002040F66A1621
:10310000B14200D100BFC1F3421501F01F030126F7
:1031100006FA03F3012D02D19689334006E0022D11
:1031200002D1168A334001E0968A33400C12012600
:1031300006FA04F41688344013B10CB1012000E003
:10314000002070BD10B50022002340F66A14A14291
:1031500000D100BF0A1201249440A3B2DC430480D2
:1031600010BD00000038014000440040004800400D
:10317000004C00400050004010B50446FA4884421C
:1031800008D101214015FEF79BFE00216015FEF7D6
:1031900097FE17E0F548844208D101210015FEF79B
:1031A0008FFE00212015FEF78BFE0BE0F0488442D5
:1031B00008D10121C803FEF783FE00214FF400402F
:1031C000FEF77EFE10BD30B5024600200023506899
:1031D000E84C20400D790C6844EA052420435060F7
:1031E0009068E54C2040D1E902542C434D7944EAE3
:1031F000450420439060D06A20F470000C7C641E6B
:10320000E4B2234340EA0350D06230BD00210160A4
:10321000017141718160C16001210174704721B168
:10322000826842F00102826003E0826822F00102BB
:103230008260704721B1826842F48072826003E04C
:10324000826822F480728260704710B50023CBB28E
:103250001AB144681C43446002E044689C434460E3
:1032600010BD816841F0080181607047014600206F
:103270008A6802F008020AB1012000E000207047CD
:10328000816841F0040181607047014600208A682E
:1032900002F004020AB1012000E00020704721B1D1
:1032A000826842F4A002826003E0826822F4A002F5
:1032B00082607047014600208A6802F480020AB1E9
:1032C000012000E00020704710B50A4600210023CD
:1032D000416821F46041531E41EA4331416010BD11
:1032E00021B1426842F40062426003E0426822F485
:1032F000006242607047F0B504460D460020002190
:10330000092D11DDE068A5F10A0606EB4607072640
:1033100006FA07F18843A5F10A0606EB460603FA0A
:1033200006F10843E0600CE0206905EB450707263D
:1033300006FA07F1884305EB450603FA06F1084350
:103340002061072A0FDA606B561E06EB86071F26E0
:1033500006FA07F18843561E06EB860605FA06F1C3
:103360000843606322E00D2A0FDA206BD61F06EBBC
:1033700086071F2606FA07F18843D61F06EB860646
:1033800005FA06F10843206310E0E06AA2F10D0699
:1033900006EB86071F2606FA07F18843A2F10D0601
:1033A00006EB860605FA06F10843E062F0BD21B19E
:1033B000826842F48012826003E0826822F4801204
:1033C000826070470146C86C80B2704766484C30D6
:1033D0000068704721B1426842F48062426003E0B5
:1033E000426822F480624260704721B1426842F430
:1033F0008052426003E0426822F48052426070478B
:103400000A460021816821F4E04111438160704740
:1034100021B1826842F40042826003E0826822F4B3
:1034200000428260704721B1826842F402128260D9
:1034300003E0826822F40212826070470146002095
:103440008A6802F400120AB1012000E000207047EF
:10345000F0B504461546002000220026092911DD9A
:10346000E068A1F10A0707EB470C072707FA0CF2FF
:103470009043A1F10A0707EB470703FA07F210434D
:10348000E0600CE0206901EB410C072707FA0CF221
:10349000904301EB410703FA07F210432061A06B50
:1034A000C0F30156EF1C06F1010CA7EB0C0707EB6C
:1034B000870C1F2707FA0CF29043EF1C06F1010C52
:1034C000A7EB0C0707EB870701FA07F21043A0638D
:1034D000F0BD10B50A4600210023816B21F4401194
:1034E000531E41EA0351816310BD08B500230093C8
:1034F0000090009B0B440093009B1A6008BD08B528
:10350000024600200090009201F12800009B184420
:1035100000900098006880B208BD0A46002141680A
:10352000164B1940114341607047416282627047F7
:103530000A460021416821F01F0111434160704794
:1035400040B109490831096841F40001064A0832CE
:10355000116007E004490831096821F40001024ABA
:10356000083211607047000000240140002801402B
:10357000003C0140FFFEF0FFFDF7F1FFFFFD3FFFC4
:103580000246002013680B400BB1012000E0002030
:103590007047CA430260704770B50246002000239E
:1035A00000240B125568CEB205EA060415681D40CA
:1035B00015B10CB1012000E0002070BD00220A12FC
:1035C000D34303607047000001684FF6FE7211405C
:1035D00001600021016041608160C1608D498842C5
:1035E00008D18C490839496841F00F01894A083AE5
:1035F00051608AE087491431884208D185490839E9
:10360000496841F0F001834A083A51607DE0814900
:103610002831884208D17F490839496841F47061EE
:103620007C4A083A516070E07A493C31884208D1BE
:1036300078490839496841F47041764A083A51603E
:1036400063E074495031884208D1724908394968A9
:1036500041F470216F4A083A516056E06D49643177
:10366000884208D16B490839496841F47001694AB8
:10367000083A516049E067497831884208D1654984
:103680000839496841F07061624A083A51603CE08B
:103690006149884206D1011F096841F00F01021FEC
:1036A000116032E05C491431884208D15A49091F3F
:1036B000096841F0F001584A121F116025E056498F
:1036C0002831884208D15449091F096841F47061C2
:1036D000514A121F116018E04F493C31884208D10D
:1036E0004D49091F096841F470414B4A121F11608E
:1036F0000BE049495031884207D14749091F096801
:1037000041F47021444A121F1160704710B5002225
:10371000026847F6F0739A430C6A8B6823430C697E
:1037200023434C6923438C692343CC6923434C6A6C
:1037300023438C6A23431A430260CB6843600B68BF
:1037400083604B68C36010BD0021016041608160EF
:10375000C160016141618161C16101624162816257
:10376000704721B1026842F00102026004E0026881
:103770004FF6FE731A40026070471AB103680B439C
:10378000036002E003688B43036070474160704749
:103790000146486880B2704701460020002201F0CF
:1037A00080531BB11C4B083B1A6802E0194B083BC5
:1037B0001A6802EA01030BB1012000E00020704703
:1037C00000F0805119B11449091F086002E0114945
:1037D00008394860704701460020002201F08053FC
:1037E0001BB10D4B083B1A6802E00A4B083B1A68F4
:1037F00002EA01030BB1012000E00020704700F055
:10380000805119B10449091F086002E001490839D3
:103810004860704708000240080402400CB50020D0
:10382000019000906C48006840F480306A4908605C
:1038300000BF6948006800F4003000900198401C07
:103840000190009818B90198B0F5A06FF1D16248C5
:10385000006800F4003010B10120009001E0002069
:1038600000900098012843D15C48006840F01000A7
:103870005A4908600846006820F0030008600846BE
:10388000006840F0020008605348406852494860B0
:103890000846406848600846406840F480604860D8
:1038A0000846406820F47C1048600846406840F4B0
:1038B000E81048600846006840F08070086000BF6B
:1038C0004548006800F000700028F9D04248406880
:1038D00020F00300404948600846406840F002007C
:1038E000486000BF3C48406800F00C000828F9D14F
:1038F0000CBD10B5FFF792FF10BD10B5364800683B
:1039000040F00100344908600846406834490840E6
:103910003149486008460068324908402E4908602D
:103920000846006820F4802008600846406820F4BB
:10393000FE0048604FF41F008860FFF7DAFF4FF089
:1039400000602949086010BD10B500210020002248
:10395000214B5B6803F00C0121B1042906D0082932
:1039600028D107E0214B224C236027E01F4B204C3D
:10397000236023E0184B5B6803F47010164B5B6800
:1039800003F48032022303EB904022B9194B4343E6
:10399000174C23600DE0104B5B6803F4003323B138
:1039A000144B4343124C236003E0104B4343104C31
:1039B000236003E00D4B0E4C236000BF00BF064B9D
:1039C0005B68C3F303130C4CE15C094B1B68CB40F1
:1039D000074C236010BD0000001002400020024090
:1039E0000000FFF8FFFFF6FE08ED00E000127A008D
:1039F0006000002000093D006400002070470000C6
:103A00000FB4044910B503AA029800F083F810BC63
:103A10005DF814FB3C00002030B505460B462A46F5
:103A200013F8014B12F8010B08B1A042F8D01CB1F9
:103A3000002802D06D1CF1E7284630BD032A40F271
:103A4000308010F0030C00F0158011F8013BBCF140
:103A5000020F624498BF11F801CB00F8013B38BF58
:103A600011F8013BA2F1040298BF00F801CB38BF66
:103A700000F8013B11F0030300F05E80083AC0F04B
:103A8000088051F8043B083A51F804CBA0E808102C
:103A9000F5E7121D5CBF51F8043B40F8043BAFF35F
:103AA0000080D20724BF11F8013B11F801CB48BFB9
:103AB00011F8012B24BF00F8013B00F801CB48BFEF
:103AC00000F8012B70474FF000020429C0F012806B
:103AD00010F0030C00F06480CCF1040CBCF1020F78
:103AE00018BF00F8012BA8BF20F8022BA1EB0C0196
:103AF00000F056B85FEAC17C24BF00F8012B00F843
:103B0000012B48BF00F8012B704770477047704782
:103B100070470000074B70B50D467B4400F06BF812
:103B20000446284600F07AF810B14FF0FF3070BD1F
:103B3000204670BDDBD5FFFF10B5203AC0F00B80EA
:103B4000B1E81850203AA0E81850B1E81850A0E8A1
:103B50001850BFF4F5AF5FEA027C24BFB1E81850FB
:103B6000A0E8185044BF18C918C0BDE810405FEA6B
:103B7000827C24BF51F8043B40F8043B08BF7047E7
:103B8000D20728BF31F8023B48BF11F8012B28BFEC
:103B900020F8023B48BF00F8012B70474FF00002AD
:103BA00000B5134694469646203922BFA0E80C5033
:103BB000A0E80C50B1F12001BFF4F7AF090728BF0E
:103BC000A0E80C5048BF0CC05DF804EB890028BF8A
:103BD00040F8042B08BF704748BF20F8022B11F0B3
:103BE000804F18BF00F8012B7047000001694A1C84
:103BF00002610878704700B58FB0CDE9013100212E
:103C0000059105497944CDE903101146684600F055
:103C10002EF80FB000BD0000E5FFFFFF007B00F0B5
:103C200080007047754600F03FF8AE4605006946D3
:103C3000534620F00700854618B020B5FCF7B2FACD
:103C4000BDE820404FF000064FF000074FF000089D
:103C50004FF0000B21F00701AC46ACE8C009ACE81E
:103C6000C009ACE8C009ACE8C0098D4670472DE931
:103C7000F04106460024D6E90170F56880463046DA
:103C800003E04146B847641C3046A8470028F8D1F5
:103C90002046BDE8F08110B50446AFF30080204611
:103CA000BDE81040FCF769BA0048704738110020A1
:103CB00076002600560026005600360102760036B1
:103CC0000000560036010076003600005600340130
:103CD00000760034000400005600320C000A000098
:103CE00000000000000000FF7600320000560031A6
:103CF000050101120436760031000056003105043A
:103D00000100191176003100005600300404010052
:103D100019760030000100560037010156003701C6
:103D200000760037000076003900005600310501AA
:103D3000011A6E0376003100000000005C3D0008AF
:103D4000000000207400000028010008D03D000899
:103D50007400002024170000440100080000000047
:103D60000000000000000000000000000000000053
:103D70000000000000000000000000000000000043
:103D80000000000000000000000000000000000033
:103D90000000000000000000000000000000000023
:103DA0000000000000000000000001020304010206
:103DB00003040607080902040608000000A24A04DA
:103DC00000000000000000000102030406070809CB
:04000005080000ED02
:00000001FF
